LINK : warning L4021: no stack segment

 Start  Stop   Length Name                   Class
 00000H 00E22H 00E23H CODERES                
 00E23H 01A1DH 00BFBH DATARES                
 01A20H 01A2FH 00010H BATARENA               
 01A30H 01A6FH 00040H BATSEG                 
 01A70H 01A7FH 00010H ENVARENA               
 01A80H 01B1FH 000A0H ENVIRONMENT            
 01B20H 026AFH 00B90H INIT                   
 026B0H 026B0H 00000H TAIL                   
 026B0H 07FA3H 058F4H TRANCODE               
 07FA4H 08458H 004B5H TRANDATA               
 08459H 09451H 00FF9H TRANSPACE              
 09460H 09460H 00000H TRANTAIL               
 09460H 09460H 00000H FOR_SEGMENT            

 Origin   Group
 0000:0   RESGROUP
 026B:0   TRANGROUP

  Address         Publics by Name

 026B:0B98       $call
 026B:1D9E       $chdir
 026B:1A57       $EXIT
 026B:0E42       $for
 026B:09FF       $if
 026B:1E04       $mkdir
 0000:1345       $M_CLS_3
 0000:26A2       $M_CLS_4
 0000:175A       $M_CLS_5
 0000:162B       $M_CLS_6
 0000:1A13       $M_CLS_7
 026B:5866       $M_CLS_8
 026B:49EC       $M_GET_MSG_ADDRESS
 026B:58C9       $M_MSGSERV_1
 026B:58EA       $M_MSGSERV_2
 026B:5E85       $M_RT
 0000:1350       $M_RT2
 026B:1E78       $rmdir
 0000:0EBF       abort_char
 026B:591C       AccDen_PTR
 026B:5AD5       ACRLF_PTR
 026B:1B08       add_name_to_environment
 026B:1AEE       add_prompt
 026B:06F3       Alloc_TPA
 026B:6277       ALLSWITCH
 0000:2366       amis_sign
 026B:65D5       APPEND_EXEC
 0000:0F5B       append_flag
 026B:481E       append_parse
 0000:0F59       append_state
 026B:65EF       arg
 026B:6273       ARG1S
 026B:6275       ARG2S
 026B:6B33       argbufptr
 026B:6270       ARGC
 026B:6277       ARGTS
 026B:2A3F       argv_calc
 026B:63CF       Arg_Buf
 026B:5A93       arg_buf_ptr
 026B:658B       ASCII
 0000:05A2       ASKEND
 0000:24BD       AUTOBAT
 026B:5913       BADBAT_PTR
 026B:3CBF       BADCDERR
 026B:5A31       BadCD_ptr
 026B:5907       badcpmes_ptr
 0000:24AE       BADCSPFL
 026B:5985       BadCurDrv
 026B:5991       BADDAT_PTR
 026B:5A51       baddev_ptr
 026B:5952       BADDRV_PTR
 0000:0E90       badfat_block
 0000:0E94       BADFAT_OP_SEG
 0000:0E8F       badfat_subst
 026B:598B       BADLAB_PTR
 026B:5A34       Badmkd_ptr
 026B:5919       BadNam_Ptr
 026B:13AB       badpath_err
 026B:5A4E       BADPMES_ptr
 026B:5A37       BADRMD_PTR
 026B:59BE       BADTIM_PTR
 026B:5A3A       BAD_ON_OFF_ptr
 026B:6D60       BatBuf
 026B:6D80       BatBufEnd
 026B:5CB3       BatBufLen
 026B:6D5E       BatBufPos
 0000:0EDB       BATCH
 026B:08CC       BatchOff
 0000:0F25       Batch_Abort
 026B:0C8E       BATCLOSE
 026B:0769       BatCom
 026B:5CA2       batext
 026B:6592       BATHAND
 026B:0CA2       BATOPEN
 026B:6587       BINARY
 026B:63A5       bits
 0000:24FB       bslash
 026B:38F0       BUILDDEST
 026B:39B0       BUILDNAME
 026B:39E0       BUILDPATH
 026B:171E       build_dir_for_chdir
 026B:16F5       build_dir_for_prompt
 026B:172F       build_dir_string
 026B:6353       bwdbuf
 026B:627B       BYTCNT
 026B:645A       bytes_free
 026B:5944       Bytmes_ptr
 0000:0F43       call_batch_flag
 0000:0F42       call_flag
 026B:0FC0       catalog
 0000:0E8E       CDEVAT
 026B:2231       cerror
 026B:6279       CFLAG
 026B:6284       charbuf
 026B:193F       chcp
 026B:626B       CHKDRV
 0000:052D       CHKSUM
 0000:24EC       CHUCKENV
 026B:180A       cls
 026B:5B38       clsstring
 026B:481A       cmd_parse
 026B:2F25       CNTRLC
 026B:62DD       COM
 026B:60B8       COMBUF
 0000:0F26       COMDRV
 026B:5C9A       comext
 026B:63AF       comma
 026B:012C       COMMAND
 0000:257B       command_c_syn
 0000:2556       command_d_syn
 0000:2562       command_e_syn
 0000:254A       command_f_syn
 0000:2587       command_m_syn
 0000:253E       command_p_syn
 0000:2590       comnd1_addr
 0000:258D       COMND1_CODE
 0000:258C       COMND1_OUTPUT
 0000:258E       comnd1_syn
 0000:258C       COMND1_TYPE
 026B:3B4F       COMPNAME
 0000:0E9C       comprmt1_block
 0000:0EA0       COMPRMT1_SEG
 0000:0EAB       COMPRMT1_SEG2
 0000:0E9B       comprmt1_subst
 026B:6BB7       comptr
 0000:0EDD       COMSPEC
 026B:5B30       comspecstr
 0000:24AF       COMSPECT
 0000:0F1D       comspec_end
 026B:65D1       comspec_flag
 0000:0E9E       comspec_print
 0000:24EF       comspstring
 026B:6271       COMSW
 026B:5B81       COMTAB
 0000:105D       COM_FCB1
 0000:1061       COM_FCB2
 0000:1059       COM_PTR
 0000:0F47       com_xlat_addr
 026B:626F       CONCAT
 026B:626E       concat_xa
 0000:1B20       CONPROC
 0000:0156       CONTC
 026B:3892       COPERR
 026B:5928       COPIED_ptr
 026B:302C       COPY
 026B:6455       copy_num
 026B:3B63       cparse
 026B:658E       CPDATE
 0000:0EB2       cpdrv
 026B:6590       CPTIME
 026B:6457       cpyflag
 026B:5971       CP_active_Ptr
 026B:5963       CP_not_all_Ptr
 026B:5955       CP_not_set_Ptr
 026B:13BC       crename
 0000:1450       critical_msg_start
 0000:0F2E       crit_err_info
 0000:0F51       crit_msg_off
 0000:0F53       crit_msg_seg
 0000:0839       CRLF
 026B:1ED9       CRLF2
 026B:1F36       CRPRINT
 026B:27D9       CTIME
 026B:5A5D       ctrlcmes_ptr
 026B:1899       ctty
 026B:59A6       curdat_mo_day
 026B:5994       CURDAT_PTR
 026B:59A4       curdat_yr
 026B:626D       CURDRV
 026B:59C6       curtim_hr_min
 026B:59C1       CURTIM_PTR
 026B:59C8       curtim_sec_hn
 0000:1636       DATARESEND
 026B:276F       DATE
 026B:6D91       date_day
 026B:6D90       date_month
 026B:6D8A       DATE_OUTPUT
 026B:6D8A       DATE_TYPE
 026B:6D8E       date_year
 026B:2737       DATINIT
 026B:5AD2       dback_ptr
 0000:0F55       dbcs_vector_addr
 026B:1BE6       delete_path
 026B:1EEE       delim
 026B:59D2       DEL_Y_N_PTR
 026B:62E0       DEST
 026B:646F       DESTBUF
 026B:627A       DestClosed
 026B:6310       destdir
 026B:6310       DESTFCB
 026B:62D4       DESTFCB2
 026B:64C6       DESTHAND
 026B:646E       destinfo
 026B:64C8       DESTISDEV
 026B:646A       Destisdir
 026B:6305       DESTNAME
 026B:646B       DESTSIZ
 026B:6275       DESTSWITCH
 026B:646C       Desttail
 026B:646A       DESTVARS
 0000:0E3E       devemes_block
 0000:0E3D       devemes_subst
 0000:0E54       DEVENAM
 0000:0E40       deve_op_off
 0000:0E42       DEVE_OP_SEG
 0000:0E4D       DEVE_OP_SEG2
 026B:5A8D       DEVWMES_ptr
 026B:6353       DIRBUF
 026B:625E       dirchar
 026B:5B08       dirdattim_ptr
 026B:5B0F       dirdat_mo_day
 026B:5B0D       dirdat_yr
 026B:63B1       dirflag
 026B:5A3D       dirhead_ptr
 026B:5936       Dirmes_ptr
 026B:5B18       dirtim_hr_min
 026B:5B1A       dirtim_sec_hn
 026B:6458       dir_num
 026B:5D89       dir_w_syn
 026B:65A5       display_ioctl
 026B:65AB       display_mode
 026B:65B3       display_width
 0000:0E23       disp_class
 026B:5AAF       disp_file_size_ptr
 026B:5ACF       Dmes_ptr
 026B:02D3       DOCOM
 026B:02D6       DOCOM1
 026B:6D9E       DRIVE_NUMBER
 026B:6D9A       DRIVE_OUTPUT
 026B:6D9A       DRIVE_TYPE
 026B:6D9B       DRIVE_VALUE
 026B:20B3       DRVBAD
 0000:0E3C       DRVLET
 0000:0E26       drvnum_block
 0000:0E28       drvnum_op_off
 0000:0E2A       DRVNUM_OP_SEG
 0000:0E35       DRVNUM_OP_SEG2
 0000:0E25       drvnum_subst
 0000:05BF       DSKERR
 026B:2560       dstrlen
 0000:2514       dswitch
 026B:2EEB       ECHO
 0000:0F31       ECHOFLAG
 026B:5A79       ECHOMES_ptr
 0000:24ED       ECOMLOC
 0000:1A8E       ECOMSPEC
 026B:6596       ELCNT
 026B:6597       ELPOS
 026B:324D       EndCopy
 0000:0566       endinit
 026B:590D       ENVERR_PTR
 0000:1B20       ENVIREND
 0000:1057       envirseg
 0000:2501       EnvMax
 0000:1FC8       EnvMaximum
 0000:24FF       envsiz
 0000:24F7       equalsign
 026B:1334       erase
 0000:0E5D       err15mes_block
 0000:0E5C       err15mes_subst
 0000:0E61       ERR15_OP_SEG
 0000:0E6C       ERR15_OP_SEG2
 0000:0E77       ERR15_OP_SEG3
 0000:0ED6       ERRCD_24
 026B:1F5E       error_output
 0000:0EC9       ErrType
 0000:2513       eswitch
 026B:5ADB       eurdat_ptr
 0000:0EB4       execemes_block
 0000:0EB6       execemes_off
 0000:0EB8       execemes_seg
 0000:0EB3       execemes_subst
 026B:6181       EXECPATH
 026B:625F       EXEC_ADDR
 0000:1057       EXEC_BLOCK
 0000:014A       Exec_Wait
 026B:5C9E       exeext
 026B:6353       EXEFCB
 026B:65D0       expand_star
 0000:0F2B       EXTCOM
 0000:1765       extended_msg_start
 026B:58FB       extend_buf_off
 026B:58F6       Extend_buf_ptr
 026B:58FD       Extend_Buf_seg
 026B:58F8       Extend_buf_sub
 026B:13AE       extend_setup
 026B:218E       EXTERNAL
 0000:1A1E       extmsgend
 026B:65A4       ext_entered
 0000:0144       EXT_EXEC
 0000:2512       ext_msg
 026B:63BA       ext_open_off
 026B:63BA       ext_open_parms
 026B:63BC       ext_open_seg
 0000:0EC2       fail_char
 026B:6BB9       fbuf
 026B:1F05       fcb_to_ascz
 0000:0F3B       fFail
 026B:6282       filecnt
 026B:5AA1       file_name_ptr
 026B:6451       file_size_high
 026B:644F       file_size_low
 026B:626C       FILTYP
 026B:1C10       FIND_NAME_IN_environment
 026B:1C08       find_path
 026B:1C0D       find_prompt
 026B:64C9       FIRSTDEST
 026B:374D       FLSHFIL
 026B:20BC       FNDCOM
 026B:09F9       forerror
 0000:0F3D       FORFLAG
 026B:5A54       fornestmes_ptr
 026B:0F99       ForOff
 026B:0D15       FORPROC
 0000:0F3E       forptr
 026B:06E3       Free_TPA
 026B:627F       FRSTSRCH
 0000:24FA       fslash
 0000:0F4C       fucase_addr
 026B:5910       FULDIR_PTR
 026B:63AD       fullscr
 026B:093D       GetBatByt
 0000:0474       GETCOMDSK2
 026B:2FF9       GetDate
 026B:0552       GetKeyStroke
 026B:1637       get_ext_error_number
 026B:160B       Get_file_code_page_tag
 026B:0BCC       goto
 026B:6353       GOTOLEN
 0000:0ED8       HANDLE01
 026B:6257       HEADCALL
 0000:24A0       icondev
 026B:62D5       ID
 026B:62D4       IDLEN
 026B:0B23       iferlev
 026B:0AB6       ifexists
 0000:0F3C       IFFlag
 026B:0A5F       ifnot
 026B:626C       IFNOTFLAG
 026B:5B65       IFTAB
 026B:6C3B       if_not_count
 0000:0EC1       ignore_char
 026B:5A5A       INBDEV_ptr
 026B:6585       INEXACT
 0000:24E0       INITADD
 0000:250D       initend
 0000:0FAD       InitFlag
 0000:229D       init_contc_specialcase
 0000:250B       init_parse
 026B:5925       inornot_ptr
 0000:1053       INPIPEPTR
 026B:6D3E       INTERNATVARS
 0000:2517       INTERNAT_INFO
 0000:02B8       INT_2E
 0000:0ECA       INT_2E_RET
 026B:5A90       inval_path_ptr
 026B:5982       inv_code_page
 0000:0F24       In_Batch
 026B:2463       IOSET
 0000:0F33       IO_SAVE
 0000:0882       ITESTKANJ
 026B:5ADE       japdat_ptr
 0000:24CE       KAUTOBAT
 026B:65EE       KPARSE
 026B:6BB5       last_arg
 0000:24F8       lcasea
 0000:24F9       lcasez
 026B:6280       lincnt
 026B:6281       linlen
 026B:65B5       linperpag
 0000:04DE       LOADCOM
 0000:0EDA       LOADING
 0000:02E9       lodcom
 0000:0355       LODCOM1
 026B:5922       LOSTERR_ptr
 0000:1069       LTPA
 026B:645E       major_ver_num
 026B:5B21       MD_exists_ptr
 026B:64CA       MELCOPY
 026B:64CB       MELSTART
 0000:0F27       MEMSIZ
 026B:6460       minor_ver_num
 026B:1C71       move_name
 026B:2599       move_to_srcbuf
 026B:58F5       Msg_Cont_Flag
 026B:58F4       msg_disp_class
 026B:65D2       msg_flag
 026B:65D3       msg_numb
 0000:08BF       MSG_SERV_ST
 0000:1067       MYSEG
 0000:106F       MYSEG1
 0000:1073       MYSEG2
 026B:5916       NEEDBAT_PTR
 0000:0F40       NEST
 026B:59B5       newdat_format
 026B:59B0       NEWDAT_PTR
 026B:59CF       NEWTIM_PTR
 0000:0F44       next_batch
 026B:597F       NLSFUNC_Ptr
 026B:02E1       NOPIPEPROC
 026B:590A       NOSPACE_PTR
 026B:2DDF       notest2
 026B:6586       NOWRITE
 0000:0EC4       no_char
 026B:5CB5       no_values
 0000:0F46       NULLFLAG
 026B:5A4B       nulpath_ptr
 0000:0E24       number_subst
 0000:2595       num_positionals
 026B:627D       NXTADD
 0000:2071       Nxtstr
 026B:658D       objcnt
 026B:5A87       offmes_ptr
 026B:1561       okvolarg
 0000:2503       oldenv
 0000:1079       olderrno
 0000:0ED2       OldTerm
 0000:2597       old_parse_ptr
 026B:6462       one_char_val
 026B:5A8A       onmes_ptr
 0000:1055       OUTPIPEPTR
 026B:0527       output_batch_name
 026B:591F       overwr_ptr
 0000:0ED0       PARENT
 026B:626F       PARM1
 026B:6270       PARM2
 026B:6D86       parse1_addr
 026B:6D83       PARSE1_CODE
 026B:6D82       PARSE1_OUTPUT
 026B:6D84       parse1_syn
 026B:6D82       parse1_type
 026B:2915       parseline
 0000:2515       parsemes_ptr
 026B:5CDE       PARSE_BREAK
 026B:5D01       parse_chcp
 026B:5D5F       parse_chdir
 026B:1AA1       parse_check_eol
 0000:2517       parse_command
 026B:5D97       parse_ctty
 026B:5D20       parse_date
 026B:5D73       parse_dir
 026B:5D68       parse_erase
 026B:63B2       parse_last
 026B:5D56       parse_mrdir
 0000:1636       parse_msg_start
 026B:5D8C       parse_rename
 026B:5D32       parse_time
 026B:5D44       parse_vol
 026B:1AB8       parse_with_msg
 0000:2507       pars_msg_off
 0000:2509       pars_msg_seg
 026B:175E       path
 026B:1F78       pathchrcmp
 026B:63A7       pathcnt
 026B:1F89       pathcrunch
 026B:6BE4       pathinfo
 026B:63A9       pathpos
 0000:1A80       PATHSTRING
 026B:63AB       PATHSW
 026B:2BC7       Path_Crunch
 026B:2A4B       path_search
 026B:5B24       PATH_TEXT
 026B:1327       Pause
 026B:5988       pausemes_ptr
 0000:0F36       PERMCOM
 026B:2449       PGetarg
 0000:0FB0       PIPE1
 0000:0FB3       pipe1t
 0000:0FC0       PIPE2
 0000:0FC3       pipe2t
 026B:25E1       PIPEDEL
 026B:5A57       PIPEEMES_PTR
 026B:2601       PIPEERRSYN
 0000:0FAF       PIPEFILES
 0000:0FAE       PIPEFLAG
 026B:285A       PipeOff
 026B:2680       PIPEPROC
 026B:262B       PIPEPROCSTRT
 0000:0FD0       PIPEPTR
 0000:0FD2       PIPESTR
 026B:658C       PLUS
 026B:63B0       plus_comma
 0000:24DF       PRDATTM
 026B:2237       PRESCAN
 026B:4826       printf_crlf
 026B:4822       printf_init
 0000:24E4       print_add
 026B:16DA       print_b
 026B:16C4       print_back
 026B:16DC       print_char
 026B:2FDF       PRINT_DATE
 026B:16EB       print_drive
 026B:16CA       print_eq
 026B:65D6       print_err_flag
 026B:16CE       print_esc
 026B:16D2       print_g
 026B:16D6       print_l
 026B:1670       PRINT_PROMPT
 026B:2872       PRINT_TIME
 026B:1657       print_version
 026B:04DF       PromptBat
 026B:5AF3       promptdat_moday
 026B:5AE1       promptdat_ptr
 026B:5AF1       promptdat_yr
 026B:5B3D       prompt_table
 026B:5B29       PROMPT_TEXT
 026B:5AFF       promtim_hr_min
 026B:5AFA       promtim_ptr
 026B:5B01       promtim_sec_hn
 026B:6BEA       psep_char
 026B:6263       RCH_ADDR
 026B:626C       RDEOF
 0000:106C       RDIRCHAR
 026B:0572       READBAT
 0000:08BF       READ_DISK_PROC
 0000:0EC5       RemMsg
 026B:5904       renerr_ptr
 0000:007F       RESCOM
 0000:2511       resetenv
 0000:08A7       reset_msg_pointers
 0000:107B       resmsgend
 0000:022F       ResPipeOff
 026B:6259       RESSEG
 0000:0F35       RESTDIR
 0000:1075       ResTest
 0000:047A       RestHand
 026B:1D91       RestUDir
 026B:1D84       restudir1
 0000:0DA6       RES_CODE_END
 0000:1077       RES_TPA
 0000:0F2C       RETCODE
 0000:0EC0       retry_char
 026B:6204       RE_INSTR
 0000:0F5D       RE_OUTSTR
 0000:0F5C       RE_OUT_APP
 026B:6465       ROM_CALL
 026B:6468       ROM_CS
 026B:0471       ROM_EXEC
 026B:6466       ROM_IP
 026B:03F8       ROM_SCAN
 0000:083C       RPRINT
 0000:0F2F       rsrc_xa_seg
 0000:0E23       rstack
 0000:106B       RSWITCHAR
 026B:2D78       Save_Args
 0000:0ECE       SAVE_PDB
 0000:0455       SavHand
 026B:1EB3       savudir
 026B:1EB6       savudir1
 026B:652C       SCANBUF
 026B:1EE6       scanoff
 026B:1C9E       scan_double_null
 026B:1CB8       scasb2
 0000:24FD       scswitch
 026B:6399       SDIRBUF
 026B:2C3C       search
 026B:6BEB       search_best
 026B:6BEC       search_best_buf
 026B:6BF9       search_curdir_buf
 026B:6C39       search_error
 026B:2CBB       Search_Ftype
 026B:38D6       SETASC
 026B:23CB       setpath
 026B:25D7       SETREST
 026B:25D5       SETREST1
 0000:0305       SetSize
 026B:3B33       SETSTARS
 026B:4B2D       SETSTDINOFF
 026B:4B14       SETSTDINON
 026B:4B5F       SETSTDOUTOFF
 026B:4B46       SETSTDOUTON
 026B:1ACC       setup_parse_error_msg
 0000:0547       SETVECT
 026B:1627       set_ext_error_msg
 026B:15DC       set_file_code_page
 026B:0B51       shift
 0000:0F37       SINGLECOM
 026B:25C0       SINGLETEST
 026B:0B84       SkipDelim
 026B:06D2       SkipToEOL
 026B:6598       SKPDEL
 026B:2E47       slashp_erase
 026B:5CDB       slash_p_syn
 026B:6599       SOURCE
 0000:24FC       space
 026B:627A       SPECDRV
 026B:64D2       srcbuf
 026B:6529       SRCHAND
 026B:64D1       SRCINFO
 026B:652B       SRCISDEV
 026B:64CD       SRCISDIR
 026B:6583       SRCPT
 026B:64CE       SRCSIZ
 026B:64CF       SRCTAIL
 026B:64CD       SRCVARS
 026B:5F87       srcxname
 026B:63B8       src_xa_seg
 026B:63B6       src_xa_size
 026B:6D3E       STACK
 026B:6594       STARTEL
 026B:482D       std_eprintf
 026B:4835       std_printf
 026B:1D0D       store_char
 026B:2BB3       Store_PChar
 026B:1F2B       strcomp
 026B:0928       StrCpy
 026B:5ABD       string_buf_ptr
 026B:6453       string_ptr_2
 026B:2D16       strip
 026B:65D8       Subst_buffer
 0000:0F29       SUM
 0000:0F32       SUPPRESS
 026B:59D5       SUREMES_ptr
 026B:2082       SWITCH
 026B:625D       SWITCHAR
 026B:5CA6       switch_list
 026B:598E       SYNTMES_PTR
 0000:0AB1       SYSDISPMSG
 0000:096C       SYSGETMSG
 026B:63B4       system_cpage
 026B:5ACC       tab_ptr
 026B:0104       TCOMMAND
 026B:658A       TERMREAD
 026B:2487       TESTDOREIN
 026B:24CF       TESTDOREOUT
 026B:1CC0       TESTKANJ
 0000:03EC       THEADFIX
 026B:6D99       time_fraction
 026B:6D96       time_hour
 026B:6D97       time_minutes
 026B:6D92       TIME_OUTPUT
 026B:6D98       time_seconds
 026B:6D92       TIME_TYPE
 0000:03CD       tjmp
 026B:625B       TPA
 026B:6B35       tpbuf
 026B:5155       TranCodeLast
 026B:5DA9       TRANDATAEND
 0000:0F1F       TRANS
 026B:6DA2       TRANSPACEEND
 0000:26B0       TranStart
 0000:1079       TranVarEnd
 0000:1065       TRANVARS
 026B:6269       TRAN_TPA
 0000:03D1       TREMCHECK
 026B:5FDE       trgxname
 026B:256E       triageError
 0000:24E8       triage_add
 026B:2595       Triage_Init
 0000:0F23       TrnMvFlg
 0000:0F21       TRNSEG
 0000:250F       trnsize
 026B:19D5       truename
 026B:3740       TRYFLUSH
 026B:4925       Tsysgetmsg
 026B:491F       TSYSLOADMSG
 026B:146D       typefil
 0000:24FE       ucasea
 026B:6035       UCOMBUF
 026B:1CEA       upconv
 026B:5AD8       usadat_ptr
 0000:2505       usedenv
 026B:613B       USERDIR1
 026B:2F68       VERIFY
 026B:5A6B       VERIMES_ptr
 026B:59D8       vermes_ptr
 026B:164E       version
 0000:0F39       VERVAL
 026B:59FF       volmes_ptr
 026B:59F1       volmes_ptr_2
 0000:0E7E       VolName
 0000:0E8A       VOLSER
 026B:5A18       volsermes_ptr
 026B:153D       volume
 026B:6464       vol_drv
 026B:65B7       vol_ioctl_buf
 026B:65BD       vol_label
 026B:65B9       vol_serial
 026B:59AD       WeekTab
 026B:6588       WRITTEN
 026B:5CAB       xa_cp
 026B:63CD       xa_cp_length
 026B:63C0       xa_cp_out
 026B:63CB       xa_list_attr
 0000:0EC3       yes_char
 026B:6C3D       zflag

  Address         Publics by Value

 0000:007F       RESCOM
 0000:0144       EXT_EXEC
 0000:014A       Exec_Wait
 0000:0156       CONTC
 0000:022F       ResPipeOff
 0000:02B8       INT_2E
 0000:02E9       lodcom
 0000:0305       SetSize
 0000:0355       LODCOM1
 0000:03CD       tjmp
 0000:03D1       TREMCHECK
 0000:03EC       THEADFIX
 0000:0455       SavHand
 0000:0474       GETCOMDSK2
 0000:047A       RestHand
 0000:04DE       LOADCOM
 0000:052D       CHKSUM
 0000:0547       SETVECT
 0000:0566       endinit
 0000:05A2       ASKEND
 0000:05BF       DSKERR
 0000:0839       CRLF
 0000:083C       RPRINT
 0000:0882       ITESTKANJ
 0000:08A7       reset_msg_pointers
 0000:08BF       MSG_SERV_ST
 0000:08BF       READ_DISK_PROC
 0000:096C       SYSGETMSG
 0000:0AB1       SYSDISPMSG
 0000:0DA6       RES_CODE_END
 0000:0E23       rstack
 0000:0E23       disp_class
 0000:0E24       number_subst
 0000:0E25       drvnum_subst
 0000:0E26       drvnum_block
 0000:0E28       drvnum_op_off
 0000:0E2A       DRVNUM_OP_SEG
 0000:0E35       DRVNUM_OP_SEG2
 0000:0E3C       DRVLET
 0000:0E3D       devemes_subst
 0000:0E3E       devemes_block
 0000:0E40       deve_op_off
 0000:0E42       DEVE_OP_SEG
 0000:0E4D       DEVE_OP_SEG2
 0000:0E54       DEVENAM
 0000:0E5C       err15mes_subst
 0000:0E5D       err15mes_block
 0000:0E61       ERR15_OP_SEG
 0000:0E6C       ERR15_OP_SEG2
 0000:0E77       ERR15_OP_SEG3
 0000:0E7E       VolName
 0000:0E8A       VOLSER
 0000:0E8E       CDEVAT
 0000:0E8F       badfat_subst
 0000:0E90       badfat_block
 0000:0E94       BADFAT_OP_SEG
 0000:0E9B       comprmt1_subst
 0000:0E9C       comprmt1_block
 0000:0E9E       comspec_print
 0000:0EA0       COMPRMT1_SEG
 0000:0EAB       COMPRMT1_SEG2
 0000:0EB2       cpdrv
 0000:0EB3       execemes_subst
 0000:0EB4       execemes_block
 0000:0EB6       execemes_off
 0000:0EB8       execemes_seg
 0000:0EBF       abort_char
 0000:0EC0       retry_char
 0000:0EC1       ignore_char
 0000:0EC2       fail_char
 0000:0EC3       yes_char
 0000:0EC4       no_char
 0000:0EC5       RemMsg
 0000:0EC9       ErrType
 0000:0ECA       INT_2E_RET
 0000:0ECE       SAVE_PDB
 0000:0ED0       PARENT
 0000:0ED2       OldTerm
 0000:0ED6       ERRCD_24
 0000:0ED8       HANDLE01
 0000:0EDA       LOADING
 0000:0EDB       BATCH
 0000:0EDD       COMSPEC
 0000:0F1D       comspec_end
 0000:0F1F       TRANS
 0000:0F21       TRNSEG
 0000:0F23       TrnMvFlg
 0000:0F24       In_Batch
 0000:0F25       Batch_Abort
 0000:0F26       COMDRV
 0000:0F27       MEMSIZ
 0000:0F29       SUM
 0000:0F2B       EXTCOM
 0000:0F2C       RETCODE
 0000:0F2E       crit_err_info
 0000:0F2F       rsrc_xa_seg
 0000:0F31       ECHOFLAG
 0000:0F32       SUPPRESS
 0000:0F33       IO_SAVE
 0000:0F35       RESTDIR
 0000:0F36       PERMCOM
 0000:0F37       SINGLECOM
 0000:0F39       VERVAL
 0000:0F3B       fFail
 0000:0F3C       IFFlag
 0000:0F3D       FORFLAG
 0000:0F3E       forptr
 0000:0F40       NEST
 0000:0F42       call_flag
 0000:0F43       call_batch_flag
 0000:0F44       next_batch
 0000:0F46       NULLFLAG
 0000:0F47       com_xlat_addr
 0000:0F4C       fucase_addr
 0000:0F51       crit_msg_off
 0000:0F53       crit_msg_seg
 0000:0F55       dbcs_vector_addr
 0000:0F59       append_state
 0000:0F5B       append_flag
 0000:0F5C       RE_OUT_APP
 0000:0F5D       RE_OUTSTR
 0000:0FAD       InitFlag
 0000:0FAE       PIPEFLAG
 0000:0FAF       PIPEFILES
 0000:0FB0       PIPE1
 0000:0FB3       pipe1t
 0000:0FC0       PIPE2
 0000:0FC3       pipe2t
 0000:0FD0       PIPEPTR
 0000:0FD2       PIPESTR
 0000:1053       INPIPEPTR
 0000:1055       OUTPIPEPTR
 0000:1057       EXEC_BLOCK
 0000:1057       envirseg
 0000:1059       COM_PTR
 0000:105D       COM_FCB1
 0000:1061       COM_FCB2
 0000:1065       TRANVARS
 0000:1067       MYSEG
 0000:1069       LTPA
 0000:106B       RSWITCHAR
 0000:106C       RDIRCHAR
 0000:106F       MYSEG1
 0000:1073       MYSEG2
 0000:1075       ResTest
 0000:1077       RES_TPA
 0000:1079       TranVarEnd
 0000:1079       olderrno
 0000:107B       resmsgend
 0000:1345       $M_CLS_3
 0000:1350       $M_RT2
 0000:1450       critical_msg_start
 0000:162B       $M_CLS_6
 0000:1636       parse_msg_start
 0000:1636       DATARESEND
 0000:175A       $M_CLS_5
 0000:1765       extended_msg_start
 0000:1A13       $M_CLS_7
 0000:1A1E       extmsgend
 0000:1A80       PATHSTRING
 0000:1A8E       ECOMSPEC
 0000:1B20       ENVIREND
 0000:1B20       CONPROC
 0000:1FC8       EnvMaximum
 0000:2071       Nxtstr
 0000:229D       init_contc_specialcase
 0000:2366       amis_sign
 0000:24A0       icondev
 0000:24AE       BADCSPFL
 0000:24AF       COMSPECT
 0000:24BD       AUTOBAT
 0000:24CE       KAUTOBAT
 0000:24DF       PRDATTM
 0000:24E0       INITADD
 0000:24E4       print_add
 0000:24E8       triage_add
 0000:24EC       CHUCKENV
 0000:24ED       ECOMLOC
 0000:24EF       comspstring
 0000:24F7       equalsign
 0000:24F8       lcasea
 0000:24F9       lcasez
 0000:24FA       fslash
 0000:24FB       bslash
 0000:24FC       space
 0000:24FD       scswitch
 0000:24FE       ucasea
 0000:24FF       envsiz
 0000:2501       EnvMax
 0000:2503       oldenv
 0000:2505       usedenv
 0000:2507       pars_msg_off
 0000:2509       pars_msg_seg
 0000:250B       init_parse
 0000:250D       initend
 0000:250F       trnsize
 0000:2511       resetenv
 0000:2512       ext_msg
 0000:2513       eswitch
 0000:2514       dswitch
 0000:2515       parsemes_ptr
 0000:2517       parse_command
 0000:2517       INTERNAT_INFO
 0000:253E       command_p_syn
 0000:254A       command_f_syn
 0000:2556       command_d_syn
 0000:2562       command_e_syn
 0000:257B       command_c_syn
 0000:2587       command_m_syn
 0000:258C       COMND1_OUTPUT
 0000:258C       COMND1_TYPE
 0000:258D       COMND1_CODE
 0000:258E       comnd1_syn
 0000:2590       comnd1_addr
 0000:2595       num_positionals
 0000:2597       old_parse_ptr
 0000:26A2       $M_CLS_4
 0000:26B0       TranStart
 026B:0104       TCOMMAND
 026B:012C       COMMAND
 026B:02D3       DOCOM
 026B:02D6       DOCOM1
 026B:02E1       NOPIPEPROC
 026B:03F8       ROM_SCAN
 026B:0471       ROM_EXEC
 026B:04DF       PromptBat
 026B:0527       output_batch_name
 026B:0552       GetKeyStroke
 026B:0572       READBAT
 026B:06D2       SkipToEOL
 026B:06E3       Free_TPA
 026B:06F3       Alloc_TPA
 026B:0769       BatCom
 026B:08CC       BatchOff
 026B:0928       StrCpy
 026B:093D       GetBatByt
 026B:09F9       forerror
 026B:09FF       $if
 026B:0A5F       ifnot
 026B:0AB6       ifexists
 026B:0B23       iferlev
 026B:0B51       shift
 026B:0B84       SkipDelim
 026B:0B98       $call
 026B:0BCC       goto
 026B:0C8E       BATCLOSE
 026B:0CA2       BATOPEN
 026B:0D15       FORPROC
 026B:0E42       $for
 026B:0F99       ForOff
 026B:0FC0       catalog
 026B:1327       Pause
 026B:1334       erase
 026B:13AB       badpath_err
 026B:13AE       extend_setup
 026B:13BC       crename
 026B:146D       typefil
 026B:153D       volume
 026B:1561       okvolarg
 026B:15DC       set_file_code_page
 026B:160B       Get_file_code_page_tag
 026B:1627       set_ext_error_msg
 026B:1637       get_ext_error_number
 026B:164E       version
 026B:1657       print_version
 026B:1670       PRINT_PROMPT
 026B:16C4       print_back
 026B:16CA       print_eq
 026B:16CE       print_esc
 026B:16D2       print_g
 026B:16D6       print_l
 026B:16DA       print_b
 026B:16DC       print_char
 026B:16EB       print_drive
 026B:16F5       build_dir_for_prompt
 026B:171E       build_dir_for_chdir
 026B:172F       build_dir_string
 026B:175E       path
 026B:180A       cls
 026B:1899       ctty
 026B:193F       chcp
 026B:19D5       truename
 026B:1A57       $EXIT
 026B:1AA1       parse_check_eol
 026B:1AB8       parse_with_msg
 026B:1ACC       setup_parse_error_msg
 026B:1AEE       add_prompt
 026B:1B08       add_name_to_environment
 026B:1BE6       delete_path
 026B:1C08       find_path
 026B:1C0D       find_prompt
 026B:1C10       FIND_NAME_IN_environment
 026B:1C71       move_name
 026B:1C9E       scan_double_null
 026B:1CB8       scasb2
 026B:1CC0       TESTKANJ
 026B:1CEA       upconv
 026B:1D0D       store_char
 026B:1D84       restudir1
 026B:1D91       RestUDir
 026B:1D9E       $chdir
 026B:1E04       $mkdir
 026B:1E78       $rmdir
 026B:1EB3       savudir
 026B:1EB6       savudir1
 026B:1ED9       CRLF2
 026B:1EE6       scanoff
 026B:1EEE       delim
 026B:1F05       fcb_to_ascz
 026B:1F2B       strcomp
 026B:1F36       CRPRINT
 026B:1F5E       error_output
 026B:1F78       pathchrcmp
 026B:1F89       pathcrunch
 026B:2082       SWITCH
 026B:20B3       DRVBAD
 026B:20BC       FNDCOM
 026B:218E       EXTERNAL
 026B:2231       cerror
 026B:2237       PRESCAN
 026B:23CB       setpath
 026B:2449       PGetarg
 026B:2463       IOSET
 026B:2487       TESTDOREIN
 026B:24CF       TESTDOREOUT
 026B:2560       dstrlen
 026B:256E       triageError
 026B:2595       Triage_Init
 026B:2599       move_to_srcbuf
 026B:25C0       SINGLETEST
 026B:25D5       SETREST1
 026B:25D7       SETREST
 026B:25E1       PIPEDEL
 026B:2601       PIPEERRSYN
 026B:262B       PIPEPROCSTRT
 026B:2680       PIPEPROC
 026B:2737       DATINIT
 026B:276F       DATE
 026B:27D9       CTIME
 026B:285A       PipeOff
 026B:2872       PRINT_TIME
 026B:2915       parseline
 026B:2A3F       argv_calc
 026B:2A4B       path_search
 026B:2BB3       Store_PChar
 026B:2BC7       Path_Crunch
 026B:2C3C       search
 026B:2CBB       Search_Ftype
 026B:2D16       strip
 026B:2D78       Save_Args
 026B:2DDF       notest2
 026B:2E47       slashp_erase
 026B:2EEB       ECHO
 026B:2F25       CNTRLC
 026B:2F68       VERIFY
 026B:2FDF       PRINT_DATE
 026B:2FF9       GetDate
 026B:302C       COPY
 026B:324D       EndCopy
 026B:3740       TRYFLUSH
 026B:374D       FLSHFIL
 026B:3892       COPERR
 026B:38D6       SETASC
 026B:38F0       BUILDDEST
 026B:39B0       BUILDNAME
 026B:39E0       BUILDPATH
 026B:3B33       SETSTARS
 026B:3B4F       COMPNAME
 026B:3B63       cparse
 026B:3CBF       BADCDERR
 026B:481A       cmd_parse
 026B:481E       append_parse
 026B:4822       printf_init
 026B:4826       printf_crlf
 026B:482D       std_eprintf
 026B:4835       std_printf
 026B:491F       TSYSLOADMSG
 026B:4925       Tsysgetmsg
 026B:49EC       $M_GET_MSG_ADDRESS
 026B:4B14       SETSTDINON
 026B:4B2D       SETSTDINOFF
 026B:4B46       SETSTDOUTON
 026B:4B5F       SETSTDOUTOFF
 026B:5155       TranCodeLast
 026B:5866       $M_CLS_8
 026B:58C9       $M_MSGSERV_1
 026B:58EA       $M_MSGSERV_2
 026B:58F4       msg_disp_class
 026B:58F5       Msg_Cont_Flag
 026B:58F6       Extend_buf_ptr
 026B:58F8       Extend_buf_sub
 026B:58FB       extend_buf_off
 026B:58FD       Extend_Buf_seg
 026B:5904       renerr_ptr
 026B:5907       badcpmes_ptr
 026B:590A       NOSPACE_PTR
 026B:590D       ENVERR_PTR
 026B:5910       FULDIR_PTR
 026B:5913       BADBAT_PTR
 026B:5916       NEEDBAT_PTR
 026B:5919       BadNam_Ptr
 026B:591C       AccDen_PTR
 026B:591F       overwr_ptr
 026B:5922       LOSTERR_ptr
 026B:5925       inornot_ptr
 026B:5928       COPIED_ptr
 026B:5936       Dirmes_ptr
 026B:5944       Bytmes_ptr
 026B:5952       BADDRV_PTR
 026B:5955       CP_not_set_Ptr
 026B:5963       CP_not_all_Ptr
 026B:5971       CP_active_Ptr
 026B:597F       NLSFUNC_Ptr
 026B:5982       inv_code_page
 026B:5985       BadCurDrv
 026B:5988       pausemes_ptr
 026B:598B       BADLAB_PTR
 026B:598E       SYNTMES_PTR
 026B:5991       BADDAT_PTR
 026B:5994       CURDAT_PTR
 026B:59A4       curdat_yr
 026B:59A6       curdat_mo_day
 026B:59AD       WeekTab
 026B:59B0       NEWDAT_PTR
 026B:59B5       newdat_format
 026B:59BE       BADTIM_PTR
 026B:59C1       CURTIM_PTR
 026B:59C6       curtim_hr_min
 026B:59C8       curtim_sec_hn
 026B:59CF       NEWTIM_PTR
 026B:59D2       DEL_Y_N_PTR
 026B:59D5       SUREMES_ptr
 026B:59D8       vermes_ptr
 026B:59F1       volmes_ptr_2
 026B:59FF       volmes_ptr
 026B:5A18       volsermes_ptr
 026B:5A31       BadCD_ptr
 026B:5A34       Badmkd_ptr
 026B:5A37       BADRMD_PTR
 026B:5A3A       BAD_ON_OFF_ptr
 026B:5A3D       dirhead_ptr
 026B:5A4B       nulpath_ptr
 026B:5A4E       BADPMES_ptr
 026B:5A51       baddev_ptr
 026B:5A54       fornestmes_ptr
 026B:5A57       PIPEEMES_PTR
 026B:5A5A       INBDEV_ptr
 026B:5A5D       ctrlcmes_ptr
 026B:5A6B       VERIMES_ptr
 026B:5A79       ECHOMES_ptr
 026B:5A87       offmes_ptr
 026B:5A8A       onmes_ptr
 026B:5A8D       DEVWMES_ptr
 026B:5A90       inval_path_ptr
 026B:5A93       arg_buf_ptr
 026B:5AA1       file_name_ptr
 026B:5AAF       disp_file_size_ptr
 026B:5ABD       string_buf_ptr
 026B:5ACC       tab_ptr
 026B:5ACF       Dmes_ptr
 026B:5AD2       dback_ptr
 026B:5AD5       ACRLF_PTR
 026B:5AD8       usadat_ptr
 026B:5ADB       eurdat_ptr
 026B:5ADE       japdat_ptr
 026B:5AE1       promptdat_ptr
 026B:5AF1       promptdat_yr
 026B:5AF3       promptdat_moday
 026B:5AFA       promtim_ptr
 026B:5AFF       promtim_hr_min
 026B:5B01       promtim_sec_hn
 026B:5B08       dirdattim_ptr
 026B:5B0D       dirdat_yr
 026B:5B0F       dirdat_mo_day
 026B:5B18       dirtim_hr_min
 026B:5B1A       dirtim_sec_hn
 026B:5B21       MD_exists_ptr
 026B:5B24       PATH_TEXT
 026B:5B29       PROMPT_TEXT
 026B:5B30       comspecstr
 026B:5B38       clsstring
 026B:5B3D       prompt_table
 026B:5B65       IFTAB
 026B:5B81       COMTAB
 026B:5C9A       comext
 026B:5C9E       exeext
 026B:5CA2       batext
 026B:5CA6       switch_list
 026B:5CAB       xa_cp
 026B:5CB3       BatBufLen
 026B:5CB5       no_values
 026B:5CDB       slash_p_syn
 026B:5CDE       PARSE_BREAK
 026B:5D01       parse_chcp
 026B:5D20       parse_date
 026B:5D32       parse_time
 026B:5D44       parse_vol
 026B:5D56       parse_mrdir
 026B:5D5F       parse_chdir
 026B:5D68       parse_erase
 026B:5D73       parse_dir
 026B:5D89       dir_w_syn
 026B:5D8C       parse_rename
 026B:5D97       parse_ctty
 026B:5DA9       TRANDATAEND
 026B:5E85       $M_RT
 026B:5F87       srcxname
 026B:5FDE       trgxname
 026B:6035       UCOMBUF
 026B:60B8       COMBUF
 026B:613B       USERDIR1
 026B:6181       EXECPATH
 026B:6204       RE_INSTR
 026B:6257       HEADCALL
 026B:6259       RESSEG
 026B:625B       TPA
 026B:625D       SWITCHAR
 026B:625E       dirchar
 026B:625F       EXEC_ADDR
 026B:6263       RCH_ADDR
 026B:6269       TRAN_TPA
 026B:626B       CHKDRV
 026B:626C       RDEOF
 026B:626C       IFNOTFLAG
 026B:626C       FILTYP
 026B:626D       CURDRV
 026B:626E       concat_xa
 026B:626F       CONCAT
 026B:626F       PARM1
 026B:6270       ARGC
 026B:6270       PARM2
 026B:6271       COMSW
 026B:6273       ARG1S
 026B:6275       ARG2S
 026B:6275       DESTSWITCH
 026B:6277       ARGTS
 026B:6277       ALLSWITCH
 026B:6279       CFLAG
 026B:627A       SPECDRV
 026B:627A       DestClosed
 026B:627B       BYTCNT
 026B:627D       NXTADD
 026B:627F       FRSTSRCH
 026B:6280       lincnt
 026B:6281       linlen
 026B:6282       filecnt
 026B:6284       charbuf
 026B:62D4       IDLEN
 026B:62D4       DESTFCB2
 026B:62D5       ID
 026B:62DD       COM
 026B:62E0       DEST
 026B:6305       DESTNAME
 026B:6310       DESTFCB
 026B:6310       destdir
 026B:6353       EXEFCB
 026B:6353       GOTOLEN
 026B:6353       bwdbuf
 026B:6353       DIRBUF
 026B:6399       SDIRBUF
 026B:63A5       bits
 026B:63A7       pathcnt
 026B:63A9       pathpos
 026B:63AB       PATHSW
 026B:63AD       fullscr
 026B:63AF       comma
 026B:63B0       plus_comma
 026B:63B1       dirflag
 026B:63B2       parse_last
 026B:63B4       system_cpage
 026B:63B6       src_xa_size
 026B:63B8       src_xa_seg
 026B:63BA       ext_open_parms
 026B:63BA       ext_open_off
 026B:63BC       ext_open_seg
 026B:63C0       xa_cp_out
 026B:63CB       xa_list_attr
 026B:63CD       xa_cp_length
 026B:63CF       Arg_Buf
 026B:644F       file_size_low
 026B:6451       file_size_high
 026B:6453       string_ptr_2
 026B:6455       copy_num
 026B:6457       cpyflag
 026B:6458       dir_num
 026B:645A       bytes_free
 026B:645E       major_ver_num
 026B:6460       minor_ver_num
 026B:6462       one_char_val
 026B:6464       vol_drv
 026B:6465       ROM_CALL
 026B:6466       ROM_IP
 026B:6468       ROM_CS
 026B:646A       DESTVARS
 026B:646A       Destisdir
 026B:646B       DESTSIZ
 026B:646C       Desttail
 026B:646E       destinfo
 026B:646F       DESTBUF
 026B:64C6       DESTHAND
 026B:64C8       DESTISDEV
 026B:64C9       FIRSTDEST
 026B:64CA       MELCOPY
 026B:64CB       MELSTART
 026B:64CD       SRCVARS
 026B:64CD       SRCISDIR
 026B:64CE       SRCSIZ
 026B:64CF       SRCTAIL
 026B:64D1       SRCINFO
 026B:64D2       srcbuf
 026B:6529       SRCHAND
 026B:652B       SRCISDEV
 026B:652C       SCANBUF
 026B:6583       SRCPT
 026B:6585       INEXACT
 026B:6586       NOWRITE
 026B:6587       BINARY
 026B:6588       WRITTEN
 026B:658A       TERMREAD
 026B:658B       ASCII
 026B:658C       PLUS
 026B:658D       objcnt
 026B:658E       CPDATE
 026B:6590       CPTIME
 026B:6592       BATHAND
 026B:6594       STARTEL
 026B:6596       ELCNT
 026B:6597       ELPOS
 026B:6598       SKPDEL
 026B:6599       SOURCE
 026B:65A4       ext_entered
 026B:65A5       display_ioctl
 026B:65AB       display_mode
 026B:65B3       display_width
 026B:65B5       linperpag
 026B:65B7       vol_ioctl_buf
 026B:65B9       vol_serial
 026B:65BD       vol_label
 026B:65D0       expand_star
 026B:65D1       comspec_flag
 026B:65D2       msg_flag
 026B:65D3       msg_numb
 026B:65D5       APPEND_EXEC
 026B:65D6       print_err_flag
 026B:65D8       Subst_buffer
 026B:65EE       KPARSE
 026B:65EF       arg
 026B:6B33       argbufptr
 026B:6B35       tpbuf
 026B:6BB5       last_arg
 026B:6BB7       comptr
 026B:6BB9       fbuf
 026B:6BE4       pathinfo
 026B:6BEA       psep_char
 026B:6BEB       search_best
 026B:6BEC       search_best_buf
 026B:6BF9       search_curdir_buf
 026B:6C39       search_error
 026B:6C3B       if_not_count
 026B:6C3D       zflag
 026B:6D3E       INTERNATVARS
 026B:6D3E       STACK
 026B:6D5E       BatBufPos
 026B:6D60       BatBuf
 026B:6D80       BatBufEnd
 026B:6D82       parse1_type
 026B:6D82       PARSE1_OUTPUT
 026B:6D83       PARSE1_CODE
 026B:6D84       parse1_syn
 026B:6D86       parse1_addr
 026B:6D8A       DATE_TYPE
 026B:6D8A       DATE_OUTPUT
 026B:6D8E       date_year
 026B:6D90       date_month
 026B:6D91       date_day
 026B:6D92       TIME_OUTPUT
 026B:6D92       TIME_TYPE
 026B:6D96       time_hour
 026B:6D97       time_minutes
 026B:6D98       time_seconds
 026B:6D99       time_fraction
 026B:6D9A       DRIVE_TYPE
 026B:6D9A       DRIVE_OUTPUT
 026B:6D9B       DRIVE_VALUE
 026B:6D9E       DRIVE_NUMBER
 026B:6DA2       TRANSPACEEND

Program entry point at 0000:0100
